:1000000002009CC0D0C0E0D2D381BC32FFFFFFFF12
:10001000FFFFFFC0D0C0E0C2D3818032FFFFFFFFEF
:10002000FFFFFF10981002005FFFFF32FFFFFFFF8E
:10003000FFFFFF020B51C0D0C0E0D2D3C2D4E523F2
:10004000A824C3985002241014600C748028F8E58A
:1000500099F6052453240F10990FD0E0D0D032C068
:10006000D0C0E0D2D3C2D480EEA825E526C39870D4
:1000700006D29CC20780E3749028F8E6F59905251E
:1000800053250F80D5E548B40005C296C29522B429
:100090000105D296C29522D296D29522C2D3C2D45D
:1000A00074105587700302017A79F878FFE4F61826
:1000B000D9FC7581BD90400FE4F07405F0F09040DC
:1000C0000E7408F090400DE4F090400F7404F0E4DA
:1000D000904000F0904001F0904002F0904003F01A
:1000E000904004F0904005F0904006F0904007F0FA
:1000F000904008F0904009F090400AF090400BF0DA
:1001000090400CF0D21012177B601D12103E78B890
:10011000760078B59007C37903E493F6A308D9F97C
:10012000752730121715801278B59007C37903E44C
:1001300093FAE6B502D5A308D9F512156E601175CC
:1001400090BF75A08075B0FFC3C2F743870280EAF5
:10015000C2B4D2B478B8E6601078B9E6F54DF54F80
:1001600078BAE6F54EF550D20D5387EF2094081279
:1001700015B1D2060203FF02045BC212D211C2B44F
:10018000D2B47548007581BD300D04D2A8D2AF300D
:10019000B0FDD2061215DD53883F758B00758DA614
:1001A00053890F438910D28E308FFDC28E121609EB
:1001B000600E120574C211300F031204A902045B11
:1001C000D212C211C29412100E120F2D120F8312EE
:1001D000053010140B100AF7100C0280F5020454BD
:1001E00012101AC2B41215B1C2B5C200C29C780A6C
:1001F00010000280FBD8F9740C1216B3E533121606
:10020000B3740D1216B32007FD78007900D8FED91B
:10021000FCD2B50204540D35204D485A20524543B6
:10022000455054494F4E2053454C45435445442076
:1002300020202020202020202020202020202000DE
:100240000D3130204D485A20524543455054494FB6
:100250004E2053454C454354454420202020202027
:10026000202020202020202020000D3135204D4846
:100270005A20524543455054494F4E2053454C4512
:1002800043544544202020202020202020202020CE
:10029000202020000D414C4C20434F554E545320FC
:1002A00048415645204245454E20434C4541524524
:1002B00044202020202020202020202020000D501D
:1002C0005245535320434C45415220414741494EEA
:1002D000204F52204F54484552204B455920544FEF
:1002E0002041424F525420000D5757562054494D3B
:1002F00045204D4541535552454D454E5420494E9C
:100300002050524F47524553532020202020202078
:1003100020000D5757562054494D4520434F525207
:10032000454354494F4E2052454345495645442084
:100330002020202020202020202020000D4E4F2093
:100340005757562054494D4520434F525245435428
:10035000494F4E2057415320524543454956454445
:100360002020202020002007FD78007900D8FED929
:10037000FCD2B522D29C121690C29CB4550122B474
:10038000560122B4582C9002BEC2B51216E81203D0
:1003900066D29C121690C29CB4581012103E900265
:1003A00094C2B51216E812036680C9D0E0D0E0020C
:1003B0000444B424BF12100E9002E8C2B51216E82D
:1003C000120366C29C120F2D120F8375480012058E
:1003D0003010090B100508100AF4100C1280F2C23C
:1003E000DE900312C2B51216E8120366020374C24D
:1003F000DE90033CC2B51216E8120366020374C213
:1004000096C295900216C2B51216E8120366120340
:1004100074B45602802ED296C295900240C2B51294
:1004200016E8120366120374B4560280D2D296D232
:100430009590026AC2B51216E8120366120374B4EC
:10044000560280D2C2B5121060120366120374B451
:1004500056AD80D9C2ACC2AA12171575A800300DCE
:100460000D7581BD12047F12047FD2A8D2AF7590A2
:10047000BF75A08075B0FFC3C2F743870280DC322E
:10048000C2D4C2B4D2B4D211C2AA1204A830B0FDF0
:10049000D2AA200B101215DD120574C211D0E0D0C3
:1004A000D0200F052202056F32C0D0C0E0D2D3C2E7
:1004B000D4C20FD2AA30B2FDD2A8801DC2D430114E
:1004C0000CD20FC2A812052FD0E0D0D022D2AAC2DF
:1004D000A812052F30B2FDD2A8200D03020514E5A5
:1004E0004FC39401F54FE5509400F5504004454F3B
:1004F0007038854D4F854E50200E2F20DE2CD20EA9
:1005000012100EC2D3120F2D120F83754800120560
:1005100030200D04C2A8800E10090B100508100A27
:10052000ED100C0280EBC20EC2DED0E0D0D0223241
:10053000754902120085C200C201C202C203C20490
:100540007A007B007C07DAFEDBFCDCFA120FFCE5AC
:10055000F9FAE5E9F9E5F9B502F5740029F5EC7465
:10056000643AF5FCC2DAC2DC75DC4975DE2122850D
:100570004C81800785814CD20BD2AA78227912C097
:1005800000C001121609D001D000700ED8F1D9EFC9
:10059000D2B4C20B22854C8180F6121690209A05A7
:1005A00075180080D6B527E8C2B4120B029005E09A
:1005B0007800790AFAE893B50202800508D9F68036
:1005C000CF1205EA309CFDD2B453883F758B00757D
:1005D0008DA053890FD28E308FFDD2B5C28E809BF5
:1005E0004D564449215341747362E828289005F11F
:1005F0007302061502073F0207600207A30207C93C
:100600000207F70208A30208C60209A4020A2E0282
:10061000059502069D120B02B421F7300D0A120B4C
:100620002F9007311216E822120B2F90072A12166C
:10063000E8309CFDD2B453883F758B00758DA05374
:10064000890FD28E308FFDD2B5C28E12100E120FCE
:100650002D120F83754800C294120530100929101D
:100660000508100AF4100C1880F27518017519327B
:10067000D294120B2F740D1216B3740A1216B322F1
:1006800075180175193080E875180175193180E009
:10069000C294120B2F9007311216E88025B4310E48
:1006A000120B02B4211975480012008580E2B432A1
:1006B0002D120B02B4210875480112008580D10269
:1006C0000595309CFDD2B453883F758B00758DA085
:1006D00053890FD28E308FFDD2B5C28E80FEB433D7
:1006E0000E120B02B4217675480212008580A1B467
:1006F000341F120B02B42165C2A8C20DC20FC20E74
:1007000090400E7400F0120B2F9007311216E88003
:10071000B1B43549120B02B4214390400E7408F075
:10072000120B2F9007311216E822313830330D0AA0
:1007300000303030300D0A00303030310D0A0012F8
:100740000B02B42118120B2F9007381216E87518F7
:100750000120100575192B800375192D22020595AE
:10076000120B02B43210120B02B421F17518067983
:10077000191211B3801CB43110120B02B421DE75B2
:10078000180679191211608009B430D1120B02B425
:1007900021CB120B2F1216FC740D1216B3740A1211
:1007A00016B322120B02B421B4120B2F9007B3120E
:1007B00016E82231302048414E4441522020353441
:1007C0003141203234350D0A00120B2F740D1216F0
:1007D000B3740A1216B32278187906C000C0011249
:1007E0000B02D001D000F608D9F1227518000205DD
:1007F000950D0A00020595120B02B43313120B0279
:10080000B421F1120B2F9007F11216E812103E22BC
:10081000B4321B1207D7120B02B421CF120B2F9048
:1008200007F11216E8791812123D75180022B4313A
:100830001D1207D7120B02B421B1120B2F9007F132
:100840001216E87918121206751800C21022B43078
:100850004F120AADEF4E701FC2A8C20DC20EC20FDA
:10086000754D00754E00120B2F9007F11216E878A7
:10087000B876001217152278B876FFD20DC20EEEA8
:10088000F54DF54F78B9F6EF78BAF6F550F54ED24A
:10089000A8120B2F9007F11216E812171522D0E0BC
:1008A000020595120B02C0E0120B02B421F0D0E059
:1008B000F527120B2F740D1216B3740A1216B31209
:1008C000171522020595120B02B421F7C2B590400C
:1008D00000E0F8E0B5000280FAC29C53883F758BB7
:1008E00000758D1053890FD28E308FFDC28EE52793
:1008F00090161093F599D207C2AF904005E05403CB
:1009000024301216B3904004E0540F24301216B372
:10091000904003E0540724301216B3904002E05494
:100920000F24301216B3904001E054072430121601
:10093000B3904000E0540F24301216B3742C1216FA
:10094000B3904009E0540124301216B3904008E0FF
:10095000540F24301216B3904007E0540324301291
:1009600016B3904006E0540F24301216B390400B9B
:10097000E0540F24301216B390400AE0D2AF540F67
:1009800024301216B3740D1216B3740A1216B32261
:1009900002059540354D3D004031304D3D00403120
:1009A000354D3D00120B02B421E6120B2F90104B77
:1009B0001216E878A0E6FC08E6FD1210EB1216FC11
:1009C00074201216B39009931216E878A8E6FC0872
:1009D000E6FD78AEE62CFC08E63DFD1210EB1216A3
:1009E000FC74201216B39009981216E878AAE6FC57
:1009F00008E6FD78B0E62CFC08E63DFD1210EB128F
:100A000016FC74201216B390099E1216E878ACE614
:100A1000FC08E6FD78B2E62CFC08E63DFD1210EB82
:100A20001216FC740D1216B3740A1216B322120BAE
:100A300002F9C3943A4008742049C394578004E9EA
:100A4000C39430540FC4C0E0120B02F9C3943A406F
:100A500008742049C394578004E9C39430540FF9B3
:100A6000D0E049F8E6C0E0120B02B4213BD0E0F937
:100A7000C4540F2430FAC3943A400474072AFAEAA3
:100A8000F519E9540F2430FAC3943A400474072A44
:100A9000FAEAF51A751802120B2F1216FC740D12D1
:100AA00016B3740A1216B322D0E00205957F007EB9
:100AB000007518007819C007C006C000120B02D0DC
:100AC00000D006D007B42103E51822B42E0605187D
:100AD000F60880E2FA742FC39A50DBEAC3943A40D6
:100AE0000280D30518EAF608EE75F00AA4FEABF012
:100AF000EF75F00AA42BFFEAC394302EFEE43FFF0B
:100B000080B4783A7903C000C001121609D001D030
:100B1000007007D8F1D9EF020595121690309A01AE
:100B200022C2AF00854C81751800D2AF02057BC28E
:100B30009CC2B553883F758B00758D1053890FD2B9
:100B40008E308FFDC28EE52790161093F599D2074F
:100B500022C0D0C0E0C083C082C0F0C2D3D2D410C3
:100B6000DC03020C08200315200212E5EE2400F538
:100B7000EDE5FE3405F5FD75DD49020E9D20970B70
:100B800085EE2885FE29D201020C0885EE2A85FE15
:100B90002BE52AC39528FAE52B95297006C3743CEA
:100BA0009A500FC201100202805E75DE0075DE21D0
:100BB00080B9E52A2400F5ECE52B3464F5FC10023D
:100BC00012300106C201C204803E052D200414D259
:100BD000048035D203D204752D01752C01753200C5
:100BE000753DFFC3E52A9528FAE52B9529C313FB2C
:100BF000EA132480FAEB3400FBE5282AF5EAEB350A
:100C000029F5FAC2D875DA4910D803020E9DE5EA33
:100C10002480F5EAE5FA3400F5FAC201052CE52C4A
:100C2000B4140BE52D20970104F52E020E9DB4326D
:100C30000BE52D20970104F52F020E9DB4500BE516
:100C40002D20970104F530020E9DB464FAE52D20A5
:100C5000970104F531752C00752D00C3940B5026B7
:100C60007402C3952E4014E532C53DB4FF0DE53244
:100C7000600614C3953E7003020D77020D840102D5
:100C8000040810204080E53254F80303032434F8AC
:100C9000900C7EE532540793FAE531C3941D501849
:100CA0007417C3952F40D4E52EC3940C40CDEAF4BD
:100CB00056F6020D77020D84E531C3943850147452
:100CC00035C3953040EFE52FC3942A40E8EA46F655
:100CD000020D77E531C3945350DBE530C3944840AF
:100CE000D4E532F53E20131ED21385484B75DB0048
:100CF000753330E5EA2400F5EBE5FA3432F5FBC252
:100D0000D975DB498063200860E5EAC395EBFAE515
:100D1000FA95FBFB400DEAC39480EB94014018C2A6
:100D2000138046EA2480FAEB3401400BFBEA24806E
:100D3000FAEB3430FB80DF30122DD21475DA0075F7
:100D4000DE0075DC0075DD00C2D8C2DCC2DAC2DBB1
:100D5000E5EA2400F5EBE5FA3432F5FBC2D975DBA0
:100D600049753330020F22D208E532C3943B400765
:100D7000E53DB4FF55800DE53204F532C39446508D
:100D800003020E9DD54903020EA2C200C201C20297
:100D9000C203C20475DA0075DE0075DC0075DD0083
:100DA000C2D8C2DCC2DAC2DBE5F9FAE5E9F9E5F955
:100DB000B512F5740029F5EC74643AF5FCC2DAC298
:100DC000DC75DC4975DE21020EE4FAE532C39A04D3
:100DD000C0E0C200740A12112DF545740F12112DD6
:100DE000F544741412112DF543741912112DF542A6
:100DF000741E12112DF541742312112DF540742823
:100E000012112DF53FD0E075F00A84AAF0BA000E59
:100E1000B4063D754739754635120F928003020DB1
:100E200084D205C20975DA0075DE0075DC0075DD57
:100E300000C2D8C2DCC2DAC2DBE5EA2400F5EBE589
:100E4000FA3432F5FBC2D975DB49121278020F224F
:100E5000754730C0E02430F546D0E0B4050280C1CB
:100E6000B40105120FA880B9B40413E54445454503
:100E700042454345414540B430A7053F80A3B403F4
:100E800010E544454545424543B43095120FDF8097
:100E900090E5444545B43089120FBE808410DA02D3
:100EA000802275DA0075DE0075DC0075DD00C2D8C1
:100EB000C2DCC2DAC2DB0548E548B403037548006A
:100EC000D20A802010DB02801B20970EE5ED240063
:100ED000F5EDE5FD3405F5FD800A75DD0075DE31C3
:100EE000D202803E10D9028039E5EB2400F5EBE513
:100EF000FB3432F5FBD200300505120F928023300F
:100F0000130AE53304B43A027430F533E54A04F5C4
:100F10004AB4780E300807D20912133F8004D20C6D
:100F2000C20AD0F0D082D083D0E0D0D032C2AF009D
:100F3000C200C201C202C203C204C205C208C20981
:100F4000C20AC20CC213C2DEC28C758CB8758AB8D4
:100F50005389F043890275DA0075DB0075DC007592
:100F6000DD0075DE00C2D8C2D9C2DAC2DBC2DCD273
:100F7000BE75F90075E90075D904D2DED28CD2AE07
:100F8000D2AF2275EB0075FB32C2D975DB49754AC9
:100F90000022E54704F547B43A44754730E5460476
:100FA000F546B43639754630E54504F545B43A2E74
:100FB000754530E54404F544B43623754430E543C3
:100FC00004F543B4340DE542B43213754330754231
:100FD00030800CB43A08754330E54204F54222E50E
:100FE0004104F541B43AF7754130E54004F540B4A9
:100FF0003AEC754030E53F04F53F80E2E5485403A4
:101000002324A2F8E62401F608E63400F62278A0AC
:10101000E62401F608E63400F622E54B54032324C7
:10102000A8F8E62401F608E63400F622E548540361
:101030002324AEF8E62401F608E63400F62278A070
:101040007914E4F608D9FC12171522545249455375
:101050003D00354D3D0031304D3D0031354D3D00B9
:10106000C2B5740D1216B390104B1216E878A0E6B4
:10107000FC08E6FD1210EB1216FC74201216B39059
:1010800010521216E878A8E6FC08E6FD78AEE62CC9
:10109000FC08E63DFD1210EB1216FC74201216B38C
:1010A0009010561216E878AAE6FC08E6FD78B0E63D
:1010B0002CFC08E63DFD1210EB1216FC74201216F3
:1010C000B390105B1216E878ACE6FC08E6FD78B247
:1010D000E62CFC08E63DFD1210EB1216FC2007FD85
:1010E00078007904D8FED9FCD2B522791D7A05ECB6
:1010F00075F00A84FCAEF0ED75F00A84FDAFF07473
:1011000006A42E75F00A842CFC743025F0F719EF34
:1011100075F019A42CFCE43DFD4C6006DAD175187D
:101120000522DA047518052277301980F5253DF877
:10113000C3953E4005E8C3943CF8E854F803030324
:101140002434C854077006E6540F243022FBE6F915
:1011500008E6FAEA13FAE913F9DBF8540F2430220F
:1011600090400D7401F0E030E104E4F080F2C2AF91
:10117000904005E054032430F709904004E0540FF8
:101180002430F709904003E054072430F7099040D9
:1011900002E0540F2430F709904001E05407243056
:1011A000F709904000E0540F2430F790400DE4F030
:1011B000D2AF2290400D7401F0E030E104E4F08001
:1011C000F2C2AF904009E054012430F70990400882
:1011D000E0540F2430F709904007E054032430F71F
:1011E00009904006E0540F2430F70990400BE0547A
:1011F0000F2430F70990400AE0540F2430F7904054
:101200000DE4F0D2AF22C2AF90400F7405F0F0743D
:1012100004F0904005E7F009904004E7F0099040A1
:1012200003E7F009904002E7F009904001E7F00978
:10123000904000E7F090400DE4F0D2AF2290400DD6
:101240007401F0E030E104E4F080F2C2AF904009B4
:10125000E7F009904008E7F009904007E7F00990AF
:101260004006E7F00990400BE7F00990400AE7F0EC
:1012700090400DE4F0D2AF2290400F7405F074045A
:10128000F0794212120679181211B3E51CC394309A
:1012900075F00AA4F9E51DC394302979FF6006753D
:1012A000F00484A9F0E53FC3943075F00AA4FAE590
:1012B00040C394302A75F00AA4FAABF0E541C39418
:1012C000302AFAE43BFB901333780C7C01E970235D
:1012D000EAC3941FFDEB94004030FB4D602C0CEDF5
:1012E000FAC3941DFDEB94004020FB4D601CA3A3AA
:1012F000EDFA0CEAFDE493CDC39DFDEB9400400AAA
:10130000FB4D6006EDFA0CA3D8E9EC75F00A8424D5
:1013100030F518743025F0F519EA75F00A84243098
:10132000F51A743025F0F51B791812123D12102CA5
:10133000C210221F1C1F1E1F1E1F1F1E1F1E1F90BC
:10134000400F7405F07404F07918121160E533C38E
:10135000951D700412101A225002240AB40504D2FA
:101360001080F1F8C39405500512137880E6740AD2
:10137000C398F81213D380DCE51D28F51DC3943AF9
:10138000404B2430F51DE51C04F51CB4363F751C9C
:1013900030E51B04F51BB43A34751B30E51A04F52F
:1013A0001AB43629751A30E51904F519B43A0775D7
:1013B000193005188017B43414E518B4320F7518B5
:1013C00030751930791812120612142B227918125E
:1013D000120622E51DC398F51DC394305047243AE8
:1013E000F51DE51C14F51CB42F3B751C35E51B14CD
:1013F000F51BB42F30751B39E51A14F51AB42F25D7
:10140000751A35E51914F519B42F1A751939E51837
:1014100014F518B42F0F7518327519337918121284
:10142000061214F62279181212062279181211B334
:10143000E518C3943075F00AA4F8E519C394302870
:10144000F8E51B04F51BC8B40243C8B4392FE51AEC
:10145000B4320280030214F0E51CC3943075F00A24
:10146000A4F9E51DC3943029600875F00484E5F003
:10147000607E751933751A30751B318073B43A70FC
:10148000751B30E51A04F51AB4336580E5C8B43A23
:1014900008751B30E51A04F51AE51AC3943075F087
:1014A0000AA4F9E51BC3943029F9E890133393C3D8
:1014B00099503D08E8B40D24751830751931751A26
:1014C00030751B31E51D04F51DB43A24751D30E55A
:1014D0001C04F51CB43A19751C30801475F00A848C
:1014E0002430F518743025F0F519751A30751B3154
:1014F000791812123D2279181211B3E51B14F51B4D
:10150000B42F65751B39E51A14F51AB42F5AE5186E
:10151000C3943075F00AA4F8E519C3943028147008
:1015200002740CF875F00A842430F518743025F034
:10153000F519E890133393F9C375F00A842430F554
:101540001A743025F0F51BE8B4021DE51CC3943075
:1015500075F00AA4F9E51DC3943029600B75F004F9
:1015600084E5F07003751B39791812123D22900042
:10157000007A237B197C087D847E007F00E493A39E
:10158000F97808E913F9EF13FFEE13FE5006EE6C3D
:10159000FEEF6DFFD8EDDAE5DBE3EE4F22540F24CA
:1015A00030F8C394394004E80216B37407280216D1
:1015B000B3C2AF00C2CA752300752400752500753B
:1015C0002600C20775987075CA8075CBFB75CC80F4
:1015D00075CDFB75C830D2CAD2AFD2AC22C2AF0033
:1015E000C2CA752300752400752500752600C20740
:1015F00075987075CAE075CBFE75CCE075CDFE753B
:10160000C830D2CAD2AFD2AC22A823E524C39822D4
:10161000008182038405068788090A8B0C8D8E0F52
:10162000901112931495961718999A1B9C1D1E9F42
:10163000A02122A324A5A62728A9AA2BAC2D2EAF32
:1016400030B1B233B43536B7B8393ABB3CBDBE3F22
:10165000C04142C344C5C64748C9CA4BCC4D4ECF12
:1016600050D1D253D45556D7D8595ADB5CDDDE5F02
:1016700060E1E263E46566E7E8696AEB6CEDEE6FF2
:10168000F07172F374F5F67778F9FA7BFC7D7EFFE2
:1016900012160960FBE5232480F8E6052353230F87
:1016A00020060122901610F8547F93B50003547F52
:1016B00022E42230060490161093C2AF00200707E0
:1016C000D207F599D2AF22FAE525A826C398500291
:1016D0002410147005D2AFEA80E0749028F8EAF67E
:1016E000052653260FD2AF22E493B4000122C08214
:1016F000C0831216B3D083D082A380ECAA187819C5
:10170000E4B5020122E6C000C0021216B3D002D036
:101710000008DAF122E52778B4F678BCE4F608F69A
:101720001217B878BCEEF608EFF67800D8FED8FEAF
:101730007485C2931217E2D2937485C2931217E292
:10174000D2937484C2931217E2D2937B0F78A0795C
:1017500083E9C2931217E2740829F9E61217E20826
:10176000E61217E208D293DBE87481C2931217E203
:1017700078007912D8FED9FCD293227800D8FED80E
:10178000FE7485C2931217E2D2937485C293121726
:10179000E2D2937B0F78A07987E9C2931217E274A3
:1017A0000829F91217EFF6081217EFF608D293DBA3
:1017B000E878B4E6F527800078A07A1E9084087E49
:1017C000007F00E6FD7B08ED13FDEF13FFEE13FE37
:1017D0005008EE6582FEEF6583FFDBEB08DAE4EE8E
:1017E0004F227A0833B39291C292D292DAF6227AD9
:1017F00008A290B333C292D292DAF622284329206B
:10180000436F7079726967687420313939302C20E0
:10181000313939312048414E4441522C20494E4300
:101820002EEF99FFFFFFFFFFFFFFFFFFFFFFFFFF0F
:10183000FFFFFFFFFFFFFFFFFFFFFFFFFFFFFFFFB8
:10184000FFFFFFFFFFFFFFFFFFFFFFFFFFFFFFFFA8
:10185000FFFFFFFFFFFFFFFFFFFFFFFFFFFFFFFF98
:10186000FFFFFFFFFFFFFFFFFFFFFFFFFFFFFFFF88
:00000001FF
